Archive member included       because of file (symbol)

C:/agb/lib/libagbsyscall.a(AgbSysCpuSet.o)
                              Main.o (CpuSet)
C:/agb/lib/libagbsyscall.a(AgbSysRegisterRamReset.o)
                              Main.o (RegisterRamReset)
C:/agb/lib/libagbsyscall.a(AgbSysVBlankIntrWait.o)
                              Main.o (VBlankIntrWait)
C:/agb/lib/libagbbackup.a(AgbDacs.o)
                              DacsTest.o (SetDacsTimerIntr)
C:/agb/lib/libagbbackup.a(AgbDacs_wram.o)
                              C:/agb/lib/libagbbackup.a(AgbDacs.o) (PollingDacsSR)
C:/agb/lib/libagbbackup.a(AgbEeprom.o)
                              MemDump.o (eeprom)
C:/agb/lib/libagbbackup.a(AgbFlash.o)
                              FlashTest.o (ProgramFlashSector)
C:/agb/lib/libagbbackup.a(AgbFl_LE39FW512.o)
                              C:/agb/lib/libagbbackup.a(AgbFlash.o) (defaultFlash)
C:/agb/lib/libagbbackup.a(AgbFl_MX29L512.o)
                              C:/agb/lib/libagbbackup.a(AgbFlash.o) (MX29L512)
C:/agb/lib/libagbbackup.a(AgbFl_AT29LV512.o)
                              C:/agb/lib/libagbbackup.a(AgbFlash.o) (AT29LV512_lib)
C:/agb/lib/libagbbackup.a(AgbSram.o)
                              MemDump.o (ReadSram)
mylib/libmyfunc.a(bg.o)       Main.o (InitBg)
mylib/libmyfunc.a(obj.o)      Main.o (SetOamBuffer)
mylib/libmyfunc.a(sound.o)    mylib/libmyfunc.a(obj.o) (snd_csrMove)
mylib/libmyfunc.a(stdSub.o)   Main.o (key)
mylib/libmyfunc.a(sincos.o)   mylib/libmyfunc.a(stdSub.o) (SIN)
C:\PROGRA~1\CYGNUS\THUMBELF-000512\H-I686-CYGWIN32\BIN/../lib/gcc-lib/thumb-elf/2.9-arm-000512/libgcc.a(_call_via_rX.o)
                              C:/agb/lib/libagbbackup.a(AgbDacs.o) (_call_via_r0)
C:\PROGRA~1\CYGNUS\THUMBELF-000512\H-I686-CYGWIN32\BIN/../lib/gcc-lib/thumb-elf/2.9-arm-000512/libgcc.a(_divsi3.o)
                              sound/m4aLib.o (__divsi3)
C:\PROGRA~1\CYGNUS\THUMBELF-000512\H-I686-CYGWIN32\BIN/../lib/gcc-lib/thumb-elf/2.9-arm-000512/libgcc.a(_dvmd_tls.o)
                              C:\PROGRA~1\CYGNUS\THUMBELF-000512\H-I686-CYGWIN32\BIN/../lib/gcc-lib/thumb-elf/2.9-arm-000512/libgcc.a(_divsi3.o) (__div0)
C:\PROGRA~1\CYGNUS\THUMBELF-000512\H-I686-CYGWIN32\BIN/../lib/gcc-lib/thumb-elf/2.9-arm-000512/libgcc.a(_udivsi3.o)
                              mylib/libmyfunc.a(bg.o) (__udivsi3)
C:\PROGRA~1\CYGNUS\THUMBELF-000512\H-I686-CYGWIN32\BIN/../lib/gcc-lib/thumb-elf/2.9-arm-000512/libgcc.a(_umodsi3.o)
                              mylib/libmyfunc.a(bg.o) (__umodsi3)

Allocating common symbols
Common symbol       size              file

m4a_sound           0xfb0             sound/m4aLib.o
kaku2               0x4               C:/agb/lib/libagbbackup.a(AgbDacs.o)
old_dacs_remainder  0x4               DacsTest.o
eeprom              0x4               C:/agb/lib/libagbbackup.a(AgbEeprom.o)
dacs_remainder      0x4               C:/agb/lib/libagbbackup.a(AgbDacs.o)
IntrTable           0x38              Main.o
kaku1               0x4               C:/agb/lib/libagbbackup.a(AgbDacs.o)
m4a_mplay000        0x40              sound/SoundDat.o
ExtMPlyJmpTbl       0x90              sound/m4aLib.o
old_flash_remainder
                    0x4               FlashTest.o
ActiveProcess       0x4               Main.o
dacs                0x4               C:/agb/lib/libagbbackup.a(AgbDacs.o)
pollingSR           0x4               C:/agb/lib/libagbbackup.a(AgbFlash.o)
m4a_cgbchn          0x100             sound/m4aLib.o
m4a_mplay001        0x40              sound/SoundDat.o
m4a_mplay002        0x40              sound/SoundDat.o
ProgramFlashSector  0x4               C:/agb/lib/libagbbackup.a(AgbFlash.o)
flash               0x4               C:/agb/lib/libagbbackup.a(AgbFlash.o)
key                 0x1c              mylib/libmyfunc.a(stdSub.o)
flash_remainder     0x4               C:/agb/lib/libagbbackup.a(AgbFlash.o)
dacs_timeoutFlag    0x4               C:/agb/lib/libagbbackup.a(AgbDacs.o)
m4a_memacc_area     0x10              sound/SoundDat.o
m4a_mplay003        0x40              sound/SoundDat.o
EraseFlashChip      0x4               C:/agb/lib/libagbbackup.a(AgbFlash.o)
dacs_timer_count    0x4               C:/agb/lib/libagbbackup.a(AgbDacs.o)
EraseFlashSector    0x4               C:/agb/lib/libagbbackup.a(AgbFlash.o)

Memory Configuration

Name             Origin             Length             Attributes
*default*        0x00000000         0xffffffff

Linker script and memory map

LOAD crt0.o
LOAD Main.o
LOAD Data.o
LOAD MemDump.o
LOAD SramTest.o
LOAD FlashTest.o
LOAD EepromTest.o
LOAD DacsTest.o
LOAD sound/m4aLib.o
LOAD sound/SoundDat.o
LOAD sound/synbsc2.o
LOAD sound/brassc3.o
LOAD sound/mutetpc4.o
LOAD sound/cutgtg3.o
LOAD sound/sawg3.o
LOAD sound/sinec3.o
LOAD sound/revcym.o
LOAD sound/wario.o
LOAD C:/agb/lib/libagbsyscall.a
LOAD C:/agb/lib/libisagbprn.a
LOAD C:/agb/lib/libagbbackup.a
LOAD mylib/libmyfunc.a
LOAD C:\PROGRA~1\CYGNUS\THUMBELF-000512\H-I686-CYGWIN32\BIN/../lib/gcc-lib/thumb-elf/2.9-arm-000512/libgcc.a
LOAD C:\PROGRA~1\CYGNUS\THUMBELF-000512\H-I686-CYGWIN32\BIN/../lib/gcc-lib/thumb-elf/2.9-arm-000512/../../../../thumb-elf/lib/libg.a
LOAD C:\PROGRA~1\CYGNUS\THUMBELF-000512\H-I686-CYGWIN32\BIN/../lib/gcc-lib/thumb-elf/2.9-arm-000512/../../../../thumb-elf/lib/libc.a
LOAD C:\PROGRA~1\CYGNUS\THUMBELF-000512\H-I686-CYGWIN32\BIN/../lib/gcc-lib/thumb-elf/2.9-arm-000512/libgcc.a
Address of section .text set to 0x8000000
Address of section .bss set to 0x3000000
                0x00008000                .=0x8000

.interp
 *(.interp)

.hash
 *(.hash)

.dynsym
 *(.dynsym)

.dynstr
 *(.dynstr)

.gnu.version
 *(.gnu.version)

.gnu.version_d
 *(.gnu.version_d)

.gnu.version_r
 *(.gnu.version_r)

.rel.text
 *(.rel.text)
 *(.rel.text.*)
 *(.rel.gnu.linkonce.t*)

.rela.text
 *(.rela.text)
 *(.rela.text.*)
 *(.rela.gnu.linkonce.t*)

.rel.data
 *(.rel.data)
 *(.rel.data.*)
 *(.rel.gnu.linkonce.d*)

.rela.data
 *(.rela.data)
 *(.rela.data.*)
 *(.rela.gnu.linkonce.d*)

.rel.rodata
 *(.rel.rodata)
 *(.rel.rodata.*)
 *(.rel.gnu.linkonce.r*)

.rela.rodata
 *(.rela.rodata)
 *(.rela.rodata.*)
 *(.rela.gnu.linkonce.r*)

.rel.got
 *(.rel.got)

.rela.got
 *(.rela.got)

.rel.ctors
 *(.rel.ctors)

.rela.ctors
 *(.rela.ctors)

.rel.dtors
 *(.rel.dtors)

.rela.dtors
 *(.rela.dtors)

.rel.init
 *(.rel.init)

.rela.init
 *(.rela.init)

.rel.fini
 *(.rel.fini)

.rela.fini
 *(.rela.fini)

.rel.bss
 *(.rel.bss)

.rela.bss
 *(.rela.bss)

.rel.plt
 *(.rel.plt)

.rela.plt
 *(.rela.plt)

.init
 *(.init)

.plt
 *(.plt)

.text           0x08000000     0xa37c
 *(.text)
 .text          0x08000000      0x1d8 crt0.o
                0x08000000                _start
                0x080000c0                start_vector
                0x080000fc                intr_main
 .text          0x080001d8      0x428 Main.o
                0x080005f4                IntrDummy
                0x08000370                InitMainSequence
                0x08000450                MainSequence
                0x08000528                ReturnMain
                0x08000548                VblankIntr
                0x080001d8                AgbMain
 .text          0x08000600      0x6ac MemDump.o
                0x08000770                InitMemDump
                0x08000600                InitMemSelect
                0x0800069c                MemSelect
                0x08000ad8                DrawAdressLine
                0x080009ac                MemDump
                0x08000b48                DumpData
 .text          0x08000cac      0x31c SramTest.o
                0x08000e3c                WriteSramAllArea
                0x08000d70                SramTest
                0x08000cac                InitSramTest
                0x08000f1c                SetSramWritePattern
 .text          0x08000fc8      0x4c8 FlashTest.o
                0x080010ec                FlashTest
                0x080013d4                SetFlashWritePattern
                0x080011b8                ProgramFlashAllArea
                0x08000fc8                InitFlashTest
 .text          0x08001490      0x47c EepromTest.o
                0x080015a4                EepromTest
                0x08001490                InitEepromTest
                0x08001670                ProgramEepromAllArea
                0x08001850                SetEepromWritePattern
 .text          0x0800190c      0x4d8 DacsTest.o
                0x08001d34                SetDacsWritePattern
                0x0800190c                InitDacsTest
                0x08001afc                ProgramDacsAllArea
                0x08001a30                DacsTest
 .text          0x08001de4     0x2104 sound/m4aLib.o
                0x080030fc                SoundVSyncOff_rev01
                0x08002f6c                SampFreqSet_rev01
                0x08001de4                umul3232H32
                0x08002d24                MPlayExtender
                0x080030a8                SoundClear_rev01
                0x08003e7c                ply_xsust
                0x08002e60                Clear64byte_rev
                0x08003e68                ply_xdeca
                0x08002e48                MusicPlayerJumpTableCopy
                0x08003e40                ply_xtype
                0x08003a20                MPlayVolumeControl
                0x0800322c                MPlayStart_rev01
                0x0800221c                SoundMainBTM
                0x08003ed0                ply_xswee
                0x08003178                SoundVSyncOn_rev01
                0x08002ccc                m4aMPlayFadeOut
                0x080031b4                MPlayOpen_rev01
                0x080026f4                TrackStop_rev01
                0x08002ca0                m4aMPlayAllContinue
                0x08003e54                ply_xatta
                0x08003454                MidiKey2CgbFr
                0x08003ea4                ply_xiecv
                0x08002c34                m4aSongNumContinue
                0x08003bf8                MPlayLFOSpeedSet
                0x08002a5c                DummyFunc
                0x08002a7c                MPlayFadeOut
                0x08002968                ply_endtie_rev01
                0x08002c94                m4aMPlayContinue
                0x080039f8                MPlayTempoControl
                0x08003320                FadeOutBody_rev01
                0x080034fc                CgbOscOff
                0x08003de4                ply_xxx
                0x080029f8                MidiKey2fr
                0x08002b28                m4aSoundMain
                0x08003df8                ply_xwave
                0x080033a0                TrkVolPitSet_rev01
                0x08002b34                m4aSongNumStart
                0x080029d0                ply_lfos_rev01
                0x08002a60                MPlayContinue
                0x080029e4                ply_mod_rev01
                0x08003a88                MPlayPitchControl
                0x08003b64                MP_clear_modM
                0x08002494                MPlayMain_rev01
                0x08002768                ply_note_rev01
                0x08002e74                SoundInit_rev01
                0x08002b60                m4aSongNumStartOrChange
                0x08003b84                MPlayModDepthSet
                0x08002bac                m4aSongNumStartOrContinue
                0x080035b4                CgbSound
                0x080032e0                MPlayStop_rev01
                0x08003ee4                DummyFunc_rev
                0x08003dc4                ply_xcmd
                0x08003010                SoundMode_rev01
                0x08003afc                MPlayPanpotControl
                0x08002e4c                ClearChain_rev
                0x08002448                SoundVSync_rev01
                0x08002a9c                m4aSoundInit
                0x08003eb0                ply_xiecl
                0x08003ebc                ply_xleng
                0x08002cdc                m4aMPlayImmInit
                0x08003c6c                ply_memacc
                0x08001df4                SoundMain
                0x08001e78                SoundMainRAM
                0x08002c68                m4aMPlayAllStop
                0x0800354c                CgbModVol
                0x0800221c                Clear64byte
                0x08002c00                m4aSongNumStop
                0x08002284                MPlyJmpTblCopy
                0x08003e90                ply_xrele
 .text          0x08003ee8        0x4 C:/agb/lib/libagbsyscall.a(AgbSysCpuSet.o)
                0x08003ee8                CpuSet
 .text          0x08003eec        0x4 C:/agb/lib/libagbsyscall.a(AgbSysRegisterRamReset.o)
                0x08003eec                RegisterRamReset
 .text          0x08003ef0        0x8 C:/agb/lib/libagbsyscall.a(AgbSysVBlankIntrWait.o)
                0x08003ef0                VBlankIntrWait
 .text          0x08003ef8      0x684 C:/agb/lib/libagbbackup.a(AgbDacs.o)
                0x080043cc                VerifyDacs
                0x0800433c                ProgramDacsSector
                0x08004020                ReadDacsID
                0x08004458                ReadDacs
                0x08004260                ProgramDacs_NE
                0x080040c0                ControllBlockLock
                0x080044b8                ExchangeSectorToPhysAdr
                0x08004014                CheckDacsTimeout
                0x08003f6c                StartDacsTimer
                0x08003fd8                StopDacsTimer
                0x08004110                EraseDacsSector
                0x0800439c                VerifyDacsCore
                0x08003ef8                SetDacsTimerIntr
                0x08004224                ProgramDacsHword
                0x080041e8                EraseDacsChip
                0x08004038                IdentifyDacs
                0x08004510                ExchangePhysAdrToSector
                0x08004424                VerifyDacsSector
 .text          0x0800457c       0x98 C:/agb/lib/libagbbackup.a(AgbDacs_wram.o)
                0x0800457c                PollingDacsSR
                0x080045f0                DacsTimerIntr
 .text          0x08004614      0x3bc C:/agb/lib/libagbbackup.a(AgbEeprom.o)
                0x080047dc                ReadEepromDword
                0x08004718                StopEepromTimer
                0x0800467c                SetEepromTimerIntr
                0x0800475c                Dma3Transmit
                0x08004658                EepromTimerIntr
                0x08004978                VerifyEepromDword
                0x080046b4                StartEepromTimer
                0x08004614                IdentifyEeprom
                0x08004894                ProgramEepromDword
 .text          0x080049d0      0x464 C:/agb/lib/libagbbackup.a(AgbFlash.o)
                0x08004afc                FlashTimerIntr
                0x08004b58                StartFlashTimer
                0x08004c50                PollingSR_COMMON
                0x08004c14                ReadFlash1
                0x08004cdc                ReadFlash_Core
                0x08004dc0                VerifyFlashSector
                0x080049d0                ReadFlashID
                0x08004a68                IdentifyFlash
                0x08004c18                SetReadFlash1
                0x08004b20                SetFlashTimerIntr
                0x08004d7c                VerifyFlashSector_Core
                0x08004bd0                StopFlashTimer
                0x08004d00                ReadFlash
 .text          0x08004e34      0x2a8 C:/agb/lib/libagbbackup.a(AgbFl_LE39FW512.o)
                0x08004ea8                EraseFlashSector_LE
                0x08004f44                ProgramFlashByte_LE
                0x08004e34                EraseFlashChip_LE
                0x08004f7c                ProgramFlashSector_LE
                0x080050a0                VerifyFlashCoreFF
                0x080050c4                VerifyFlashErase
 .text          0x080050dc       0xa4 C:/agb/lib/libagbbackup.a(AgbFl_MX29L512.o)
                0x080050dc                ProgramFlashSector_MX
 .text          0x08005180      0x2bc C:/agb/lib/libagbbackup.a(AgbFl_AT29LV512.o)
                0x08005300                ProgramFlashSector_AT
                0x08005378                ProgramFlash4KB_AT
                0x08005180                EraseFlashChip_AT
                0x080051f0                EraseFlashSector_AT
                0x08005274                EraseFlash4KB_AT
 .text          0x0800543c      0x15c C:/agb/lib/libagbbackup.a(AgbSram.o)
                0x08005504                VerifySram_Core
                0x08005534                VerifySram
                0x080054c4                WriteSram
                0x0800543c                ReadSram_Core
                0x08005460                ReadSram
 .text          0x08005598     0x2b98 mylib/libmyfunc.a(bg.o)
                0x08007e5c                DrawUIntOnBgx
                0x0800586c                DisableBgSecurity
                0x08005c1c                GetBgxBuffer
                0x08005b38                GetBgMode
                0x0800682c                GetBgxCharBaseAdr
                0x080069f4                GetBgxAreaOver
                0x08005c90                GetBgxBuffSize
                0x08006150                GetFlameBuff
                0x0800678c                SetBgxCharBaseAdr
                0x08006b60                SetBgxPosY
                0x08006910                GetBgxPriority
                0x0800801c                DrawSIntOnBgx
                0x08007750                CheckParagraph
                0x080062f8                GetBgxScreenBaseBlock
                0x08006960                SetBgxAreaOver
                0x08006350                SetBgxScreenBaseAdr
                0x08006adc                RelativeScrollBgxPosX
                0x080064f4                SetBgxMosaicEnable
                0x08006738                GetBgxCharBaseBlock
                0x0800728c                CalcRbgxReferenceStartPos
                0x08005890                SetBgMode
                0x08006268                SetBgxScreenBaseBlock
                0x08005bcc                SetBgxBuffRenewal
                0x08006444                SetMosaicEnable
                0x08006190                SetScreenSize
                0x08006bfc                RelativeScrollBgxPosY
                0x0800754c                RotateZoomRbgx
                0x0800665c                GetBgxColorMode
                0x08006aa4                GetBgxPosX
                0x080076b0                SetParagraph
                0x080079ec                DrawAsciiStringOnBgx
                0x08005ec0                TrmScreenDataToBgxBufferByFunc
                0x08006df0                CalcRbgxAffineValue
                0x080065cc                SetBgxColorMode
                0x08006210                GetScreenSize
                0x08007d44                DrawHalfByteHexOnBgx
                0x08005fdc                ClearBgxScreenRect
                0x08005f2c                TrmScreenDataToBgxBuffer
                0x08005ccc                ClearBgxBuffer
                0x08005598                InitBg
                0x08006584                GetBgxMosaicEnable
                0x08006110                SetFlameBuff
                0x08005e0c                DmaAllBgxBuffer
                0x08007b30                DrawHexOnBgx
                0x08006c80                SetRbgxHVflip
                0x08006d00                SetRbgxTheta
                0x080066a4                SetBgxCharBaseBlock
                0x08006d54                SetRbgxMagnify
                0x08005b68                SetBgxBuffer
                0x08005d64                DmaBgxBuffer
                0x08006a40                SetBgxPosX
                0x08005c54                GetBgxBuffPointer
                0x08006bc4                GetBgxPosY
                0x08005840                EnableBgSecurity
                0x08006880                SetBgxPriority
                0x080063ec                GetBgxScreenBaseAdr
                0x08007888                DrawAsciiCharOnBgx
 .text          0x08008130      0x590 mylib/libmyfunc.a(obj.o)
                0x080081c4                SetOamBufferRenewal
                0x08008474                CheckCursorPos
                0x0800838c                SetCursorChar
                0x08008160                DmaOamBuffer
                0x080084c4                CheckCursorPosRange
                0x08008130                SetOamBuffer
                0x0800832c                DeleteCursor
                0x08008520                MoveAndAnimeCursor
                0x080081f0                SetCursorStatus
                0x08008414                GetCurosrPosOnBg
 .text          0x080086c0       0x68 mylib/libmyfunc.a(sound.o)
                0x080086c0                SetSound
 .text          0x08008728     0x1a48 mylib/libmyfunc.a(stdSub.o)
                0x08008bdc                ReadKey
                0x080094c0                DrawNowInputHexData
                0x08008e14                ClearVram
                0x08008f80                TrmCharData
                0x08008914                AddRapidKey
                0x08008c50                ChangeTask
                0x08009b0c                DrawNowToggleSwitchChar
                0x08008cc0                CalcAffineValue
                0x08008e88                ClearOam
                0x08008a54                ReadKeyPlus
                0x08008ef0                ClearPalette
                0x08008824                SetKeyRapid
                0x08008980                ShiftInterval
                0x080096bc                DrawNowSelectString
                0x08008ca8                ExecuteTask
                0x08009108                SetInputHexData
                0x080087f8                SetKeyRapidEnable
                0x08009c90                DrawNowToggleSwitchString
                0x08009f4c                DrawNowAllSetting
                0x08009e44                ClearNowAllSetting
                0x08009144                InputHexData
                0x08008728                WaitHblank
                0x08008da4                ClearWram
                0x08008948                SubRapidKey
                0x0800a060                InitSetFunc
                0x0800902c                TrmPaletteData
                0x080097b0                ToggleSwitch
                0x0800959c                SelectStrings
                0x08008788                WaitPressKey
 .text          0x0800a170       0x3c C:\PROGRA~1\CYGNUS\THUMBELF-000512\H-I686-CYGWIN32\BIN/../lib/gcc-lib/thumb-elf/2.9-arm-000512/libgcc.a(_call_via_rX.o)
                0x0800a178                _call_via_r2
                0x0800a188                _call_via_r6
                0x0800a184                _call_via_r5
                0x0800a17c                _call_via_r3
                0x0800a19c                _call_via_fp
                0x0800a190                _call_via_r8
                0x0800a18c                _call_via_r7
                0x0800a170                _call_via_r0
                0x0800a198                _call_via_sl
                0x0800a1a4                _call_via_sp
                0x0800a194                _call_via_r9
                0x0800a180                _call_via_r4
                0x0800a174                _call_via_r1
                0x0800a1a0                _call_via_ip
                0x0800a1a8                _call_via_lr
 .text          0x0800a1ac       0x94 C:\PROGRA~1\CYGNUS\THUMBELF-000512\H-I686-CYGWIN32\BIN/../lib/gcc-lib/thumb-elf/2.9-arm-000512/libgcc.a(_divsi3.o)
                0x0800a1ac                __divsi3
 .text          0x0800a240        0x4 C:\PROGRA~1\CYGNUS\THUMBELF-000512\H-I686-CYGWIN32\BIN/../lib/gcc-lib/thumb-elf/2.9-arm-000512/libgcc.a(_dvmd_tls.o)
                0x0800a240                __div0
 .text          0x0800a244       0x78 C:\PROGRA~1\CYGNUS\THUMBELF-000512\H-I686-CYGWIN32\BIN/../lib/gcc-lib/thumb-elf/2.9-arm-000512/libgcc.a(_udivsi3.o)
                0x0800a244                __udivsi3
 .text          0x0800a2bc       0xc0 C:\PROGRA~1\CYGNUS\THUMBELF-000512\H-I686-CYGWIN32\BIN/../lib/gcc-lib/thumb-elf/2.9-arm-000512/libgcc.a(_umodsi3.o)
                0x0800a2bc                __umodsi3
 *(.text.*)
 *(.stub)
 *(.gnu.warning)
 *(.gnu.linkonce.t*)
 *(.glue_7t)
 *(.glue_7)
                0x0800a37c                _etext=.
                0x0800a37c                PROVIDE (etext, .)

.fini
 *(.fini)

.rodata         0x0800a37c    0x138d4
 *(.rodata)
 .rodata        0x0800a37c      0x12c Main.o
 .rodata        0x0800a4a8     0x3200 Data.o
                0x0800a6a8                mychar
                0x0800a4a8                textPaletteData
 .rodata        0x0800d6a8      0x150 MemDump.o
 .rodata        0x0800d7f8      0x148 SramTest.o
 .rodata        0x0800d940      0x1cc FlashTest.o
 .rodata        0x0800db0c      0x174 EepromTest.o
 .rodata        0x0800dc80      0x1a8 DacsTest.o
 .rodata        0x0800de28      0x2d8 sound/m4aLib.o
                0x0800df6c                FreqTable
                0x0800e038                CgbFrTable
                0x0800de28                MPlyJmpTbl
                0x0800e08c                Cgb3vol
                0x0800deb8                ScaleTable
                0x0800e0d0                xcmd_tbl
                0x0800e09c                clock_tbl_rev01
                0x0800dfb4                CgbScTable
                0x0800e050                NoiseTable
                0x0800df9c                pcmVBtbl_rev
 .rodata        0x0800e100      0x7bc sound/SoundDat.o
                0x0800e100                voicegroup000
                0x0800e700                voicegroup002
                0x0800e700                voicegroup001
                0x0800e810                mplay_table
                0x0800e840                song_table
 .rodata        0x0800e8bc     0x1d5c sound/synbsc2.o
                0x0800e8bc                synbsc2
 .rodata        0x08010618     0x20f8 sound/brassc3.o
                0x08010618                brassc3
 .rodata        0x08012710      0xfe4 sound/mutetpc4.o
                0x08012710                mutetpc4
 .rodata        0x080136f4     0x3f1c sound/cutgtg3.o
                0x080136f4                cutgtg3
 .rodata        0x08017610       0xb4 sound/sawg3.o
                0x08017610                sawg3
 .rodata        0x080176c4      0x270 sound/sinec3.o
                0x080176c4                sinec3
 .rodata        0x08017934     0x4c7c sound/revcym.o
                0x08017934                revcym
 .rodata        0x0801c5b0      0x770 sound/wario.o
                0x0801ccfc                wario
 .rodata        0x0801cd20      0x154 C:/agb/lib/libagbbackup.a(AgbDacs.o)
                0x0801cdda                dacsErrFlag
 .rodata        0x0801ce74       0x10 C:/agb/lib/libagbbackup.a(AgbDacs_wram.o)
 .rodata        0x0801ce84       0x84 C:/agb/lib/libagbbackup.a(AgbEeprom.o)
 .rodata        0x0801cf08       0xa4 C:/agb/lib/libagbbackup.a(AgbFlash.o)
 .rodata        0x0801cfac       0x98 C:/agb/lib/libagbbackup.a(AgbFl_LE39FW512.o)
                0x0801cfc4                defaultFlash
                0x0801cff0                LE39FW512
 .rodata        0x0801d044       0x90 C:/agb/lib/libagbbackup.a(AgbFl_MX29L512.o)
                0x0801d074                MX29L512
                0x0801d0a0                MN63F805MNP
 .rodata        0x0801d0d4       0x98 C:/agb/lib/libagbbackup.a(AgbFl_AT29LV512.o)
                0x0801d0ec                AT29LV512_lib
                0x0801d118                AT29LV512_org
 .rodata        0x0801d16c       0x1c C:/agb/lib/libagbbackup.a(AgbSram.o)
 .rodata        0x0801d188      0x100 mylib/libmyfunc.a(bg.o)
 .rodata        0x0801d288       0x38 mylib/libmyfunc.a(obj.o)
 .rodata        0x0801d2c0       0xb4 mylib/libmyfunc.a(sound.o)
                0x0801d2c0                snd_csrMove
                0x0801d2d2                snd_select
                0x0801d2d8                snd_ok
                0x0801d2cc                snd_parent
                0x0801d2c6                snd_child
 .rodata        0x0801d374       0xdc mylib/libmyfunc.a(stdSub.o)
                0x0801d374                keyArray
 .rodata        0x0801d450      0x800 mylib/libmyfunc.a(sincos.o)
                0x0801d450                SIN
                0x0801d650                COS
                0x0801d850                ASIN
                0x0801da50                ACOS
 *(.rodata.*)
 *(.gnu.linkonce.r*)

.rodata1
 *(.rodata1)
                0x0801dd50                .=(ALIGN(0x100)+(.&0xff))

.data           0x0801dd50        0x0
 *(.data)
 *(.data.*)
 *(.gnu.linkonce.d*)

.data1
 *(.data1)

.ctors
 EXCLUDE_FILE ( *crtend.o )*(.ctors)
 *(SORT(.ctors.*))
 *crtend(.ctors)

.dtors
 EXCLUDE_FILE ( *crtend.o )*(.dtors)
 *(SORT(.dtors.*))
 *crtend.o(.dtors)

.got
 *(.got.plt)
 *(.got)

.dynamic
 *(.dynamic)

.sdata
 *(.sdata)
 *(.sdata.*)
                0x0801dd50                _edata=.
                0x0801dd50                PROVIDE (edata, .)
                0x0801dd50                __bss_start=.
                0x0801dd50                __bss_start__=.

.sbss
 *(.sbss)
 *(.scommon)

.bss            0x03000000     0x341c
 *(.dynbss)
 *(.bss)
 .bss           0x03000000     0x1404 Main.o
 *fill*         0x03001404        0x4
 .bss           0x03001408       0x2c MemDump.o
 .bss           0x03001434        0x4 SramTest.o
 .bss           0x03001438        0x4 FlashTest.o
 .bss           0x0300143c        0x4 EepromTest.o
 .bss           0x03001440        0x4 DacsTest.o
 *fill*         0x03001444        0x4
 .bss           0x03001448      0x5a0 sound/SoundDat.o
 .bss           0x030019e8      0x190 C:/agb/lib/libagbbackup.a(AgbDacs.o)
 .bss           0x03001b78       0x10 C:/agb/lib/libagbbackup.a(AgbEeprom.o)
 .bss           0x03001b88       0x18 C:/agb/lib/libagbbackup.a(AgbFlash.o)
 .bss           0x03001ba0      0x134 mylib/libmyfunc.a(bg.o)
 *fill*         0x03001cd4        0x4
 .bss           0x03001cd8       0x18 mylib/libmyfunc.a(obj.o)
 .bss           0x03001cf0       0x24 mylib/libmyfunc.a(stdSub.o)
 *(.bss.*)
 .bss.code      0x03001d14      0x400 sound/m4aLib.o
                0x03001d14                SoundMainBuf
 *(COMMON)
 *fill*         0x03002114        0xc
 COMMON         0x03002120       0x3c Main.o
                                  0x0 (size before relaxing)
                0x03002120                IntrTable
                0x03002158                ActiveProcess
 COMMON         0x0300215c        0x4 FlashTest.o
                                  0x0 (size before relaxing)
                0x0300215c                old_flash_remainder
 COMMON         0x03002160        0x4 DacsTest.o
                                  0x0 (size before relaxing)
                0x03002160                old_dacs_remainder
 *fill*         0x03002164        0xc
 COMMON         0x03002170     0x1140 sound/m4aLib.o
                                  0x0 (size before relaxing)
                0x03002170                m4a_sound
                0x03003120                ExtMPlyJmpTbl
                0x030031b0                m4a_cgbchn
 COMMON         0x030032b0      0x110 sound/SoundDat.o
                                  0x0 (size before relaxing)
                0x030032b0                m4a_mplay000
                0x030032f0                m4a_mplay001
                0x03003330                m4a_mplay002
                0x03003370                m4a_memacc_area
                0x03003380                m4a_mplay003
 COMMON         0x030033c0       0x18 C:/agb/lib/libagbbackup.a(AgbDacs.o)
                                  0x0 (size before relaxing)
                0x030033c0                kaku2
                0x030033c4                dacs_remainder
                0x030033c8                kaku1
                0x030033cc                dacs
                0x030033d0                dacs_timeoutFlag
                0x030033d4                dacs_timer_count
 COMMON         0x030033d8        0x4 C:/agb/lib/libagbbackup.a(AgbEeprom.o)
                                  0x0 (size before relaxing)
                0x030033d8                eeprom
 COMMON         0x030033dc       0x18 C:/agb/lib/libagbbackup.a(AgbFlash.o)
                                  0x0 (size before relaxing)
                0x030033dc                pollingSR
                0x030033e0                ProgramFlashSector
                0x030033e4                flash
                0x030033e8                flash_remainder
                0x030033ec                EraseFlashChip
                0x030033f0                EraseFlashSector
 *fill*         0x030033f4        0xc
 COMMON         0x03003400       0x1c mylib/libmyfunc.a(stdSub.o)
                                  0x0 (size before relaxing)
                0x03003400                key
                0x0300341c                .=ALIGN(0x4)
                0x0300341c                .=ALIGN(0x4)
                0x0300341c                _end=.
                0x0300341c                _bss_end__=.
                0x0300341c                __bss_end__=.
                0x0300341c                PROVIDE (end, .)

.stab
 *(.stab)

.stabstr
 *(.stabstr)

.stab.excl
 *(.stab.excl)

.stab.exclstr
 *(.stab.exclstr)

.stab.index
 *(.stab.index)

.stab.indexstr
 *(.stab.indexstr)

.comment
 *(.comment)

.debug
 *(.debug)

.line
 *(.line)

.debug_srcinfo
 *(.debug_srcinfo)

.debug_sfnames
 *(.debug_sfnames)

.debug_aranges  0x00000000      0x240
 *(.debug_aranges)
 .debug_aranges
                0x00000000       0x20 Main.o
 .debug_aranges
                0x00000020       0x20 MemDump.o
 .debug_aranges
                0x00000040       0x20 SramTest.o
 .debug_aranges
                0x00000060       0x20 FlashTest.o
 .debug_aranges
                0x00000080       0x20 EepromTest.o
 .debug_aranges
                0x000000a0       0x20 DacsTest.o
 .debug_aranges
                0x000000c0       0x20 C:/agb/lib/libagbbackup.a(AgbDacs.o)
 .debug_aranges
                0x000000e0       0x20 C:/agb/lib/libagbbackup.a(AgbDacs_wram.o)
 .debug_aranges
                0x00000100       0x20 C:/agb/lib/libagbbackup.a(AgbEeprom.o)
 .debug_aranges
                0x00000120       0x20 C:/agb/lib/libagbbackup.a(AgbFlash.o)
 .debug_aranges
                0x00000140       0x20 C:/agb/lib/libagbbackup.a(AgbFl_LE39FW512.o)
 .debug_aranges
                0x00000160       0x20 C:/agb/lib/libagbbackup.a(AgbFl_MX29L512.o)
 .debug_aranges
                0x00000180       0x20 C:/agb/lib/libagbbackup.a(AgbFl_AT29LV512.o)
 .debug_aranges
                0x000001a0       0x20 C:/agb/lib/libagbbackup.a(AgbSram.o)
 .debug_aranges
                0x000001c0       0x20 mylib/libmyfunc.a(bg.o)
 .debug_aranges
                0x000001e0       0x20 mylib/libmyfunc.a(obj.o)
 .debug_aranges
                0x00000200       0x20 mylib/libmyfunc.a(sound.o)
 .debug_aranges
                0x00000220       0x20 mylib/libmyfunc.a(stdSub.o)

.debug_pubnames
                0x00000000     0x11a8
 *(.debug_pubnames)
 .debug_pubnames
                0x00000000       0x90 Main.o
 .debug_pubnames
                0x00000090       0x31 Data.o
 .debug_pubnames
                0x000000c1       0x6e MemDump.o
 .debug_pubnames
                0x0000012f       0x5d SramTest.o
 .debug_pubnames
                0x0000018c       0x7b FlashTest.o
 .debug_pubnames
                0x00000207       0x67 EepromTest.o
 .debug_pubnames
                0x0000026e       0x76 DacsTest.o
 .debug_pubnames
                0x000002e4      0x1e1 C:/agb/lib/libagbbackup.a(AgbDacs.o)
 .debug_pubnames
                0x000004c5       0x36 C:/agb/lib/libagbbackup.a(AgbDacs_wram.o)
 .debug_pubnames
                0x000004fb       0xd6 C:/agb/lib/libagbbackup.a(AgbEeprom.o)
 .debug_pubnames
                0x000005d1      0x177 C:/agb/lib/libagbbackup.a(AgbFlash.o)
 .debug_pubnames
                0x00000748       0xbc C:/agb/lib/libagbbackup.a(AgbFl_LE39FW512.o)
 .debug_pubnames
                0x00000804       0x49 C:/agb/lib/libagbbackup.a(AgbFl_MX29L512.o)
 .debug_pubnames
                0x0000084d       0xaa C:/agb/lib/libagbbackup.a(AgbFl_AT29LV512.o)
 .debug_pubnames
                0x000008f7       0x62 C:/agb/lib/libagbbackup.a(AgbSram.o)
 .debug_pubnames
                0x00000959      0x4a1 mylib/libmyfunc.a(bg.o)
 .debug_pubnames
                0x00000dfa       0xda mylib/libmyfunc.a(obj.o)
 .debug_pubnames
                0x00000ed4       0x66 mylib/libmyfunc.a(sound.o)
 .debug_pubnames
                0x00000f3a      0x23a mylib/libmyfunc.a(stdSub.o)
 .debug_pubnames
                0x00001174       0x34 mylib/libmyfunc.a(sincos.o)

.debug_info     0x00000000    0x44725
 *(.debug_info)
 .debug_info    0x00000000     0x3cda Main.o
 .debug_info    0x00003cda     0x273b Data.o
 .debug_info    0x00006415     0x3dc6 MemDump.o
 .debug_info    0x0000a1db     0x3b28 SramTest.o
 .debug_info    0x0000dd03     0x3c91 FlashTest.o
 .debug_info    0x00011994     0x3bdd EepromTest.o
 .debug_info    0x00015571     0x3c3d DacsTest.o
 .debug_info    0x000191ae     0x3858 C:/agb/lib/libagbbackup.a(AgbDacs.o)
 .debug_info    0x0001ca06     0x2fdc C:/agb/lib/libagbbackup.a(AgbDacs_wram.o)
 .debug_info    0x0001f9e2     0x32af C:/agb/lib/libagbbackup.a(AgbEeprom.o)
 .debug_info    0x00022c91     0x3775 C:/agb/lib/libagbbackup.a(AgbFlash.o)
 .debug_info    0x00026406     0x3352 C:/agb/lib/libagbbackup.a(AgbFl_LE39FW512.o)
 .debug_info    0x00029758     0x3129 C:/agb/lib/libagbbackup.a(AgbFl_MX29L512.o)
 .debug_info    0x0002c881     0x330a C:/agb/lib/libagbbackup.a(AgbFl_AT29LV512.o)
 .debug_info    0x0002fb8b     0x306f C:/agb/lib/libagbbackup.a(AgbSram.o)
 .debug_info    0x00032bfa     0x483f mylib/libmyfunc.a(bg.o)
 .debug_info    0x00037439     0x3559 mylib/libmyfunc.a(obj.o)
 .debug_info    0x0003a992     0x3102 mylib/libmyfunc.a(sound.o)
 .debug_info    0x0003da94     0x4602 mylib/libmyfunc.a(stdSub.o)
 .debug_info    0x00042096     0x268f mylib/libmyfunc.a(sincos.o)

.debug_abbrev   0x00000000     0x2221
 *(.debug_abbrev)
 .debug_abbrev  0x00000000      0x1d1 Main.o
 .debug_abbrev  0x000001d1       0xd1 Data.o
 .debug_abbrev  0x000002a2      0x1b7 MemDump.o
 .debug_abbrev  0x00000459      0x1c4 SramTest.o
 .debug_abbrev  0x0000061d      0x1d5 FlashTest.o
 .debug_abbrev  0x000007f2      0x1c4 EepromTest.o
 .debug_abbrev  0x000009b6      0x1d5 DacsTest.o
 .debug_abbrev  0x00000b8b      0x26b C:/agb/lib/libagbbackup.a(AgbDacs.o)
 .debug_abbrev  0x00000df6      0x16d C:/agb/lib/libagbbackup.a(AgbDacs_wram.o)
 .debug_abbrev  0x00000f63      0x1cf C:/agb/lib/libagbbackup.a(AgbEeprom.o)
 .debug_abbrev  0x00001132      0x237 C:/agb/lib/libagbbackup.a(AgbFlash.o)
 .debug_abbrev  0x00001369      0x1af C:/agb/lib/libagbbackup.a(AgbFl_LE39FW512.o)
 .debug_abbrev  0x00001518      0x17e C:/agb/lib/libagbbackup.a(AgbFl_MX29L512.o)
 .debug_abbrev  0x00001696      0x1af C:/agb/lib/libagbbackup.a(AgbFl_AT29LV512.o)
 .debug_abbrev  0x00001845      0x15f C:/agb/lib/libagbbackup.a(AgbSram.o)
 .debug_abbrev  0x000019a4      0x240 mylib/libmyfunc.a(bg.o)
 .debug_abbrev  0x00001be4      0x1b8 mylib/libmyfunc.a(obj.o)
 .debug_abbrev  0x00001d9c      0x17f mylib/libmyfunc.a(sound.o)
 .debug_abbrev  0x00001f1b      0x243 mylib/libmyfunc.a(stdSub.o)
 .debug_abbrev  0x0000215e       0xc3 mylib/libmyfunc.a(sincos.o)

.debug_line     0x00000000     0x5c69
 *(.debug_line)
 .debug_line    0x00000000      0x3e8 Main.o
 .debug_line    0x000003e8      0x535 MemDump.o
 .debug_line    0x0000091d      0x324 SramTest.o
 .debug_line    0x00000c41      0x411 FlashTest.o
 .debug_line    0x00001052      0x3fa EepromTest.o
 .debug_line    0x0000144c      0x428 DacsTest.o
 .debug_line    0x00001874      0x724 C:/agb/lib/libagbbackup.a(AgbDacs.o)
 .debug_line    0x00001f98      0x159 C:/agb/lib/libagbbackup.a(AgbDacs_wram.o)
 .debug_line    0x000020f1      0x488 C:/agb/lib/libagbbackup.a(AgbEeprom.o)
 .debug_line    0x00002579      0x4f3 C:/agb/lib/libagbbackup.a(AgbFlash.o)
 .debug_line    0x00002a6c      0x38c C:/agb/lib/libagbbackup.a(AgbFl_LE39FW512.o)
 .debug_line    0x00002df8      0x169 C:/agb/lib/libagbbackup.a(AgbFl_MX29L512.o)
 .debug_line    0x00002f61      0x3b4 C:/agb/lib/libagbbackup.a(AgbFl_AT29LV512.o)
 .debug_line    0x00003315      0x1dc C:/agb/lib/libagbbackup.a(AgbSram.o)
 .debug_line    0x000034f1     0x13a5 mylib/libmyfunc.a(bg.o)
 .debug_line    0x00004896      0x37e mylib/libmyfunc.a(obj.o)
 .debug_line    0x00004c14       0xe4 mylib/libmyfunc.a(sound.o)
 .debug_line    0x00004cf8      0xf71 mylib/libmyfunc.a(stdSub.o)

.debug_frame
 *(.debug_frame)

.debug_str
 *(.debug_str)

.debug_loc
 *(.debug_loc)

.debug_macinfo
 *(.debug_macinfo)

.debug_weaknames
 *(.debug_weaknames)

.debug_funcnames
 *(.debug_funcnames)

.debug_typenames
 *(.debug_typenames)

.debug_varnames
 *(.debug_varnames)

.stack          0x00080000        0x0
                0x00080000                _stack=.
 *(.stack)
OUTPUT(blib_sample.elf elf32-littlearm)
